:100000000C945001FFFFFFFF0C94DB07FFFFFFFF85
:10001000FFFFFFFFFFFFFFFFFFFFFFFFFFFFFFFFF0
:10002000FFFFFFFFFFFFFFFFFFFFFFFFFFFFFFFFE0
:10003000FFFFFFFFFFFFFFFFFFFFFFFFFFFFFFFFD0
:10004000FFFFFFFF0C945107FFFFFFFF0C94B51C4F
:100050000C94371DFFFFFFFFFFFFFFFFFFFFFFFFB8
:10006000FFFFFFFFFFFFFFFFFFFFFFFFFFFFFFFFA0
:100070004D6F6465202020202020202044656D6F76
:100080004D6F6465202020205374616E6420427996
:100090004D6F646520496E74657272757074656425
:1000A0000000000000000000000000000000000050
:1000B0004D6F64652020502D4C696D6974696E67C1
:1000C0000000000000000000000000000000000030
:1000D0000000000000000000000000000000000020
:1000E0000000000000000000000000000000000010
:1000F0004D6F6465202020204D61782E502E502EAB
:10010000202020424954204661696C757265202088
:10011000202047726F756E64204661756C742020D4
:100120002020505631204F76657220566F6C742017
:100130002020505632204F76657220566F6C742006
:1001400020202053797374656D2045727220202021
:100150002020525844204661696C75726520202029
:1001600020205056204F76657220506F77657220A0
:10017000204772696420566F6C74204572726F72EA
:1001800020477269642046726571204572726F72F1
:10019000202054565331204661696C7572652020C9
:1001A000202054565332204661696C7572652020B8
:1001B0002020545653204661696C757265202020BA
:1001C000202020202020202020202020202020202F
:1001D0000020506C6561736520576169742E2E2E66
:1001E00020002020204165726F2D536861727020BD
:1001F00020200042617474657279204661696C75D3
:1002000072652100496E7465726E616C20546D7068
:100210002020204300542D546F74616C2020202036
:1002200020202E206800542D546F646179202020F6
:100230002020202E206800452D546F74616C2020F2
:10024000202020206B576800452D546F6461792071
:100250002020202E206B57680056707632202020F8
:10026000202020202020202056005670763120208B
:100270002020202020202020205600506F75742040
:10028000202020202020202020205700566772693F
:10029000642020202020202020202056000001FF64
:1002A000CFEFD4E0CDBFDEBFCE51D0400AEA088305
:1002B0000024EFE2F3E014E0E838F10711F00192D6
:1002C000FBCF0083E0E7F0E0A0E0B1E012E000E067
:1002D0000BBFEF39F10721F0C89531960D92F9CF98
:1002E0000E940709FFCF2227332700271127E6D0D6
:1002F00021E030E001E010E0E1D02227332709E0DF
:1003000010E0DCD0222733270BE010E0D7C08F9A13
:100310008E9A969808950027112703C000000F5F5A
:100320001F4F0A30E0E01E07C8F308954A935A931E
:100330000BC04427552703C000004F5F5F4F4A3072
:10034000E0E05E07C8F30A9580E0801790F35991CA
:10035000499108954A935A930AC04427552702C0E9
:100360004F5F5F4F4032E3E05E07D0F30A9580E0D5
:10037000801798F35991499108958F9A05E0D6DF37
:10038000979AC9DF969AC7DF979802E0E3DF9698BD
:10039000C2DF01E0DFCF969ABEDF8F9A05E0C6DFAD
:1003A0009798B9DF979AB7CF8F9A9798B4DF969AB4
:1003B000B2DF9698B0DF979A08958F9A979AABDF3D
:1003C000969AA9DF9698A7CF4A938F98A4DF969A1A
:1003D00005E0ACDF40B340789EDF969805E0A6DFED
:1003E000042F499108950E94BB1E602F8F9A48E008
:1003F00011C0862F8078A82E803811F4979A01C0FA
:10040000979889DF969A05E091DF969805E08EDF50
:10041000660F4A95442369F70C94C21E0E94BB1EC6
:1004200044278F9868E011C0969A05E07FDF440F5B
:1004300080B38078A82E803811F4416000C005E0B8
:1004400075DF969805E072DF6A95662369F7042FD9
:100450000C94C21E08950E94D71EA901A02EC88424
:10046000D9848BDF00EABFDFAFDF003811F401E091
:1004700023C08601012F1127B6DFA6DF003811F453
:1004800001E01AC00C2DAFDF9FDF602F003871F440
:1004900001E012C0FA010081A6DF96DF602F00386C
:1004A00011F401E009C04F5F5F4FAA94AA2091F7B1
:1004B00072DF01E04FDF00270C94E01E0E94C91E8E
:1004C000A22EC02E5ADF00ED8EDF7EDF003811F441
:1004D00001E013C00C2D87DF77DF003811F401E055
:1004E0000CC00A2D80DF70DF402F003811F401E0CE
:1004F00004C051DF01E02EDF00270C94D01E0E94C3
:100500009E1EC22EE02EAA2422E00027D7DF35DF70
:1005100000ED69DF59DF003811F401E01DC00E2D38
:1005200062DF52DF003891F401E016C08FE394E0FF
:10053000EA2DFF27E80FF91F008155DF45DF402F27
:10054000003811F401E008C0A394CA94CC2071F7DC
:1005500022DF03E0EBDE00270C94931E0E94D71EDF
:10056000422F5801CC2409DF00EA3DDF2DDF00389F
:1005700011F401E038C0CFDE8501012F112733DFF0
:1005800023DF003811F401E02EC0C5DE0A2D2BDF79
:100590001BDF602F003811F401E025C0EEDE01EA18
:1005A00022DF12DF602F003871F401E01CC036DF5B
:1005B000A02E88E094E0EC2DFF27E80FF91FA08221
:1005C000F3DEC3944A95413091F728DFA02E88E0EE
:1005D00094E0EC2DFF27E80FF91FA082EEDEDBDEB2
:1005E00003E0A4DE00270C94E01E0E94D71E422FD9
:1005F000A02ECC2421E0002761DFBFDE00EDF3DE7A
:10060000E3DE003811F401E030C085DE0A2DEBDEB8
:10061000DBDE003811F401E028C0AFDE01EDE3DEDF
:10062000D3DE602F003871F401E01FC0F7DEA02E8A
:100630008FE394E0EC2DFF27E80FF91FA082B4DED2
:10064000C3944A95413091F7E9DEA02E8FE394E000
:10065000EC2DFF27E80FF91FA082AFDE9CDE03E040
:1006600065DE222700272ADF00270C94E01EBC9AB3
:10067000C498B99AC19A00000000B89AC09A0000C4
:1006800000000000000022242ABA0000000009B384
:1006900003C00000000009B307FDFBCFC0988FEF37
:1006A0008ABB08958FEF8ABBBC9AC498B99AC19847
:1006B000000000000BBB00000000B89AC09A0000C8
:1006C000000000000000C09808958FEF8ABBBC9A1C
:1006D000C49AB99AC198000000000BBB000000004A
:1006E000B89AC09A0000000000000000C098089569
:1006F00008E3D8DF08EC10E00E949F1C08E3D2DF7B
:1007000008EC10E00E949F1C08E3CCDF08EC10E02E
:100710000E949F1CACDF08E3C5DFA9DF08E0C2DF51
:10072000A6DF01E0BFDFA3DF06E0BCDFA0DF0FE054
:10073000B9DF9DCF0E94C91E5901C02ECC2019F4EB
:1007400002E0B0DF02C000ECADDF91DF442706C05D
:10075000F50101915F01B9DF8ADF43954031C0F3B4
:100760000C94D01E0E94B11EA901B80128EE33E0FE
:100770008B010E94E71DC801C096FA01838728EE0D
:1007800033E08B010E94E51DB80124E630E00E94B1
:10079000E71DC801C096FA01848724E630E08B018A
:1007A0000E94E51DB8012AE030E00E94E71DC80163
:1007B000C096FA0185872AE030E08B010E94E51D92
:1007C000B801CB01C096FA0186870C94B61E0E9430
:1007D000C21D4A935A934E815F8180E492E4AFE058
:1007E000B0E00A811B812C813D81BA93AA939A9330
:1007F0008A930E94031E0A831B832C833D8380EA15
:1008000096E8A1E0B0E00A811B812C813D81BA937A
:10081000AA939A938A930E94011E1801290180E3EA
:1008200090E0A0E0B0E0280E391E4A1E5B1EFA01DF
:100830003996208280EA96E8A1E0B0E00A811B8127
:100840002C813D81BA93AA939A938A930E94031EA6
:100850000A831B832C833D8380E197E2A0E0B0E014
:100860000A811B812C813D81BA93AA939A938A9322
:100870000E94011E1801290180E390E0A0E0B0E091
:10088000280E391E4A1E5B1EFA013A96208280E12C
:1008900097E2A0E0B0E00A811B812C813D81BA93F0
:1008A000AA939A938A930E94031E0A831B832C8324
:1008B0003D8388EE93E0A0E0B0E00A811B812C81AB
:1008C0003D81BA93AA939A938A930E94011E1801BC
:1008D000290180E390E0A0E0B0E0280E391E4A1E16
:1008E0005B1EFA013B96208288EE93E0A0E0B0E028
:1008F0000A811B812C813D81BA93AA939A938A9392
:100900000E94031E0A831B832C833D8384E690E0B0
:10091000A0E0B0E00A811B812C813D81BA93AA93AB
:100920009A938A930E94011E1801290180E390E0A6
:10093000A0E0B0E0280E391E4A1E5B1EFA013C966C
:10094000208284E690E0A0E0B0E00A811B812C8147
:100950003D81BA93AA939A938A930E94031E0A83B5
:100960001B832C833D838AE090E0A0E0B0E00A8105
:100970001B812C813D81BA93AA939A938A930E94FA
:10098000011E1801290180E390E0A0E0B0E0280EEC
:10099000391E4A1E5B1EFA013D9620828AE090E0D5
:1009A000A0E0B0E00A811B812C813D81BA93AA931B
:1009B0009A938A930E94031E0A831B832C833D8390
:1009C00080E390E0A0E0B0E02A803B804C805D8036
:1009D000280E391E4A1E5B1EFA012686599149913E
:1009E000249608954A9344270BC0E42FFF27E20F73
:1009F000F31F2080E42FFF27E00FF11F2082439593
:100A0000403198F3499108950E94A71E5801442748
:100A100013C000E1122F0103100180E091E0280EC5
:100A2000391EE42FFF27E20DF31D2080E42FFF275E
:100A3000EA0DFB1D20824395403158F30C94AC1E07
:100A4000AA92A02E60972CE133E08E01CBDF9E01AD
:100A50008AE090E00091F7031091F8032F933F9301
:100A60009C010E94E71D3F912F917CDE8B85803396
:100A700039F480E28B878C85803311F480E28C8797
:100A80009E010A2D57DE6096A9900895AA92A02E85
:100A900060972BE033E08E01A5DF9E010091E50316
:100AA0001091E6035FDE8B85803361F480E28B87F3
:100AB0008C85803339F480E28C878D85803311F406
:100AC00080E28D879E010A2D35DE6096A9900895FB
:100AD000AA92A02E60972AEF32E08E0183DF9E015A
:100AE0008AE090E00091F1031091F2032F933F937D
:100AF0009C010E94E71D3F912F9134DE8B8580334E
:100B000039F480E28B878C85803311F480E28C8706
:100B10009E010A2D0FDE6096A9900895AA92A02E3C
:100B2000609729EE32E08E015DDF9E018AE090E061
:100B30000091EF031091F0032F933F939C010E94CB
:100B4000E71D3F912F910EDE8B85803339F480E2D3
:100B50008B878C85803311F480E28C879E010A2D6F
:100B6000E9DD6096A9900895AA92A02E609728EDDD
:100B700032E08E0137DF9E010091CC031091CD034E
:100B8000F1DD2C8429862D842A862E842C868EE203
:100B90008B878BE68D8787E58E878985803311F477
:100BA00080E289879E010A2DC5DD6096A99008958F
:100BB000AA92BA92A02E629727EC32E08E010E5FC5
:100BC0001F4F10DFCE010296998388832091D903AD
:100BD0003091DA030091D7031091D803F8DD2B840C
:100BE00029862C842A862D842B862E842C862F847D
:100BF0002D8628882E868BE68F8787E5888B8985CA
:100C00008033B1F480E289878A85803389F480E279
:100C10008A878B85803361F480E28B878C85803373
:100C200039F480E28C878D85803311F480E28D87E2
:100C30009E012E5F3F4F0A2D7DDD6296B990A990EF
:100C40000895AA92A02E609726EB32E08E01CADEAC
:100C50009E010091CF031091D00384DD8B858033FA
:100C600039F480E28B878C85803311F480E28C87A5
:100C70002B842A862C842B862D842C868EE28D87CD
:100C80009E010A2D57DD6096A9900895AA92A02E84
:100C9000629725EA32E08E010E5F1F4FA3DECE0180
:100CA0000296998388832091D4033091D5030091D3
:100CB000D2031091D3038BDD8B85803389F480E2DE
:100CC0008B878C85803361F480E28C878D858033BF
:100CD00039F480E28D878E85803311F480E28E872F
:100CE0002B842A862C842B862D842C862E842D867C
:100CF0002F842E868EE28F879E012E5F3F4F0A2D16
:100D000019DD6296A9900895AA924A93A02E609741
:100D100044278091DF039091E0038030E0E89E0754
:100D200038F0805090489093E0038093DF034AEAC4
:100D300024E932E08E0156DE9E018AE090E00091C7
:100D4000DF031091E0032F933F939C010E94E71D66
:100D50003F912F9107DD80E78B878C85803311F4DD
:100D600080E28C874A3A11F48DE28C879E010A2D2D
:100D7000E1DC60964991A9900895AA92CA92A02EAA
:100D800060978091DD039091DE038F709070C82E84
:100D9000C0923C04282F8E0137DE9E010A2DCADC4A
:100DA0006096C990A9900895AA924A93A02E609740
:100DB000442714C000E11A2D0103100180E991E0DD
:100DC000280E391EE42FFF27E20DF31D2080CE01EF
:100DD000E42FFF27E80FF91F20824395403150F39D
:100DE0009E010027A7DC442708C0CE01E42FFF277F
:100DF000E80FF91F80E2808343954031B0F39E01F4
:100E000001E098DC60964991A9900895AA924A93CE
:100E1000A02E6097442714C000E11A2D0103100191
:100E200080EF91E0280E391EE42FFF27E20DF31D1D
:100E30002080CE01E42FFF27E80FF91F2082439581
:100E4000403150F39E01002775DC60964991A990CE
:100E50000895609723E832E08E01C4DD9E010027EB
:100E600069DC60960895609722E732E08E01BADD72
:100E70009E0100275FDC21E632E08E01B3DD9E019A
:100E800001E058DC60960895AA92A02E609720E5B4
:100E900032E08E01A7DD9E010A2D4CDC6096A99000
:100EA00008952A923A928A939A93AA93EA932FB634
:100EB0002A9286EC82BF80918404909185040196E9
:100EC0009093850480938404883EE3E09E07C9F5EF
:100ED0002224332430928504209284048091870454
:100EE0008F5F80938704809158048F5F80935804AC
:100EF00080918704853038F02092870480913803F0
:100F000081608093380320905604222029F0822D9E
:100F100081508093560408C08B988AB780688ABF36
:100F20008BB780688BBF939A20905B04222021F0BE
:100F3000822D815080935B04809137038160809380
:100F4000370320905A04222039F0822D823320F476
:100F50008F5F80935A040FC080915A04823359F4F2
:100F600080913803877F80933803846080933803AF
:100F7000222420925A0420905904222039F0822DF4
:100F8000823320F48F5F809359040CC08091590400
:100F9000823341F4809137038061809337032224A8
:100FA0002092590429902FBEE991A9919991899194
:100FB0003990299018958A938FB78A938BB78F773A
:100FC0008BBF8AB780688ABF8B9A93988EE1809393
:100FD000560489918FBF8991189586EC82BF84E071
:100FE00083BF89B7826089BF89B78E7F89BF089523
:100FF0008FEF8ABB8BBB87BB88BB84BB85BB81BBA8
:1010000082BB86B987B9089522972090C803309093
:10101000C9033092340320923303209049042220E4
:1010200061F410914D0400E30103C001C0978E9656
:1010300090933B0480933A0412C010914D0400E356
:101040000103C001C097E0914904FF273197EE0FDB
:10105000FF1F8E0F9F1F90933B0480933A040E94C2
:101060002A02209033032092080420903403209217
:10107000090420903A0430903B043982288228E009
:1010800034E002E00E942B022296089522970E94EB
:101090002A0280914D04992780509A4F019790938E
:1010A0003B0480933A042AE030E00091CC03109195
:1010B000CD030E94E71D0093080420903A0430906D
:1010C0003B043982288228E034E001E00E942B02B0
:1010D000229608951A930A9322974090C60350903F
:1010E000C7032090C4033090C50330923003209290
:1010F0002F03509232034092310320920804209033
:101100003003209209042090310320920A04209099
:10111000320320920B0480914F0499270197880F86
:10112000991F880F991F8057994F90933B04809384
:101130003A040E942A0220903A0430903B043982FB
:10114000288228E034E004E00E942B0224960895CF
:10115000AA924A93402F142F12951F700AE00103A0
:10116000842F8F70A82EA00C0A2D4991A990089564
:1011700000270BC02227332703C000002F5F3F4FFB
:101180002F3FEFEF3E07C8F303950F3198F3089513
:10119000B8980000000000000000B09904C00AE008
:1011A00010E00E949F1C0000000000000000B89AA0
:1011B000C09808958DE693E0E0916C03FF27E80F57
:1011C000F91F2224208204E014C08DE693E02090D1
:1011D0006C033324280E391E210189E693E0E02FA9
:1011E000FF27E80FF91F2080F2013080320C308297
:1011F000039580916C038C5F081738F38DE693E0BC
:10120000E0916C03FF27E80FF91F008108952297F2
:10121000F894EEDEB898000000000000000011C055
:101220000AE010E00E949F1C86B38170813049F46F
:101230000AE010E00E949F1C86B38170813009F49F
:1012400001C0EECF0000000000000000B89AC09876
:10125000A8988EDF0E9478030E94330789DF0E94DE
:1012600087010E9473018C988D98949A959A00003A
:101270000000849945C0859943C004E610E00E94AF
:101280009F1C84993DC085993BC0222420923C0438
:1012900011C00E942A0210913C0402E3010319824A
:1012A000088228E034E00E942B0280913C048F5F8A
:1012B00080933C0480913C048E3958F30E942A02AA
:1012C0008DED9EE19983888328E034E003E20E945B
:1012D0002B0280EE99E09093340380933303282E01
:1012E00020920804292E209209040E942A0287EFE6
:1012F00095E09983888328E034E002E00E942B0285
:101300008C9A8D9A949A959A68DE2DE000E01FE100
:101310000E94AE02319A0E94911D209011042092E9
:10132000520426DF399A0E942B1D8B98939A85B719
:101330008C6085BF8BB780688BBF8AB780688ABF97
:10134000D8C026E100EE15E00E94AE02209008040D
:1013500020922F03209009042092300320900A0449
:101360002092310320900B042092320340903103ED
:101370005090320320902F03309030033092D803E6
:101380002092D7035092DA034092D90320900C04A4
:101390002092D60320900D0420922F0320900E045B
:1013A0002092300320900F042092310320901004EB
:1013B00020923203409031035090320320902F034B
:1013C000309030033092D3032092D2035092D50351
:1013D0004092D403209011042092330320901204F1
:1013E0002092340320903303309034033092D003A2
:1013F0002092CF03209013042092330320901404F2
:101400002092340320903303309034033092CD0384
:101410002092CC03209015042092330320901604D0
:101420002092340320903303309034033092CB0366
:101430002092CA03209017042092330320901804AE
:101440002092340320903303309034033092C90348
:101450002092C803209019042092D10320901A04EE
:1014600020922F0320901B042092300320901C0414
:101470002092310320901D042092320340903103CA
:101480005090320320902F03309030033092C503E8
:101490002092C4035092C7034092C60326E100EE97
:1014A00015E00E94AE022090080420922F032090A5
:1014B00009042092300320900A04209231032090E6
:1014C0000B0420923203409031035090320320905D
:1014D0002F03309030038090D9039090DA0360900E
:1014E000D7037090D803621473048404950409F43C
:1014F00001C027CF22242092FD0327E002E00E94B2
:10150000F50220903F0420924A042090400420924B
:1015100048042090410420924B04209043042092E0
:101520004E042090440420925004209045042092C0
:10153000510480914A048036B8F480914804803682
:1015400098F480914B04843278F481E320904E0427
:10155000821550F082E120905004821528F089E92C
:10156000209051048215D8F4222420923F0481E077
:101570008093400484E08093410485E0809342049A
:1015800081E08093430480E1809344048093450488
:1015900027E002E00E947F0281E08093FD038091BA
:1015A000FD03813081F4809136038F778093360379
:1015B000222433243092CD032092CC033092D003E6
:1015C0002092CF03F2C221E009E00E94F5022090B0
:1015D0003F0425FE28C021E00AE11FE10E94AE027F
:1015E0002090080420923C0483E0821530F480911E
:1015F0003603806880933603D8C2809136038F7794
:101600008093360380913C048F5F809308040E948E
:101610002A028AE19FE19983888328E034E001E08F
:101620000E942B02C2C22224209208040E942A0295
:101630008AE19FE19983888328E034E001E00E94F9
:101640002B02809136038F778093360322242092D9
:101650003E0426E0002711270E94AE0220900804D5
:10166000209248042090090420924B0420900B04FF
:1016700020924E0420900C042092500420900D04DF
:10168000209251040091480463DD009347040091C7
:101690004B045EDD0093490400914E0459DDA02EF9
:1016A000A0924D040091500453DDA02EA0924F044F
:1016B00026E003E00E94F50200913F0449DDA02EE0
:1016C000A0923F040091400443DDA02EA09240046C
:1016D000009142043DDDA02EA092420400914304FB
:1016E00037DDA02EA092430430904F04301609F449
:1016F00077C0032DEFDC80E08093C4038093C503A3
:101700008093C6038093C70320904F0433244090F6
:10171000430455242414350474F5342C321881E024
:10172000831530F020904D0430904204321418F0AC
:1017300080E280933E0480914F048F5F80934F043A
:1017400081E080933C040DC000914F04C3DC809184
:101750004F048F5F80934F0480913C048F5F809390
:101760003C0420904F043324409043045524241417
:10177000350454F335C020904F04309043043214A4
:1017800078F5822D8C3019F0832D813031F4209042
:101790004D0430904204321460F080E280933E04A5
:1017A00008C000914F0496DC80914F048F5F8093B6
:1017B0004F048CE020904F04821598F781E08093CD
:1017C0004F0408C000914F0485DC80914F048F5F67
:1017D00080934F042090430430904F04321490F3D0
:1017E00000915004B5DCA02EA0924F04209042043A
:1017F00030904D04321409F43FC048DC22243324D5
:101800003092CD032092CC033092D0032092CF03AC
:1018100080914D048F5F80934D042090430430905D
:101820004F043214A1F406C031DC80914D048F5F67
:1018300080934D0420904D04309042043214A0F760
:101840001BC024DC80914D048F5F80934D048FE199
:1018500020904D048215A8F781E080934D0406C0C6
:1018600015DC80914D048F5F80934D0420904204DD
:1018700030904D043214A0F321E006EF15E00E94F1
:10188000AE02209008042092390484EB821510F4F3
:101890008093390480E08093E1038093E203809396
:1018A000E3038093E403222420923C0434C022E02A
:1018B000A0903C042A2C3324022D11270050194FEC
:1018C000020D131D0E94AE022090080420923303E3
:1018D0002090090420923403209033033090340385
:1018E000442455248090E3039090E4036090E10346
:1018F0007090E203620C731C841C951C7092E203CE
:101900006092E1039092E4038092E30380913C04AF
:101910008F5F80933C042090390430903C04321453
:1019200030F244EB50E060E070E02091E30330914E
:10193000E4030091E1031091E2037A936A935A93CE
:101940004A930E94011E1093E6030093E503009161
:101950004E04FEDBA02EA0924D04209042040215FE
:10196000B1F52090430430904F04321481F520905B
:101970004004309049043214D9F0832D8F5F809356
:10198000490442DB222433243092C9032092C80345
:1019900006C0809149048F5F8093490435DB209015
:1019A00049043324409040045524241435048CF316
:1019B0002090E5033090E6034090CA035090CB039B
:1019C000420C531C5092CB034092CA03ADC080918D
:1019D0003E04803208F0A8C080914904873120F08D
:1019E00022242092490405C0809149048F5F80938E
:1019F00049040ADB222433243092C9032092C8030D
:101A0000809149048F5F809349043092CB032092E8
:101A1000CA0328EE33E00091E5031091E6030E942B
:101A2000E71D2090D6033324200E311E2092D603CA
:101A300006C0EADA809149048F5F8093490487E108
:101A4000209049048215A8F7222420924904DCDA68
:101A500020904D0430904204321408F049C0822D89
:101A60008F5F80934D0413C022242092490406C046
:101A7000CBDA809149048F5F8093490480914904B7
:101A80008831B0F380914D048F5F80934D048FE1D6
:101A900020904D04821540F781E080934D0413C0DF
:101AA00022242092490406C0AFDA809149048F5F56
:101AB00080934904809149048831B0F380914D04AA
:101AC0008F5F80934D042090420430904D04321477
:101AD00038F31CC022242092490406C095DA809174
:101AE00049048F5F80934904809149048831B0F3A1
:101AF00080914D048F5FA82EA0924D04282E332490
:101B00004090420455242414350424F322242092C6
:101B1000490406C079DA809149048F5F80934904B3
:101B2000809149048831B0F380913E04803208F4FA
:101B30003CC0222433243092C9032092C80330923F
:101B4000CD032092CC033092D0032092CF03209279
:101B50003E0481E080934D0414C022242092490465
:101B600006C052DA809149048F5F8093490487E16F
:101B7000209049048215A8F780914D048F5F8093CF
:101B80004D048FE120904D04821538F781E0809359
:101B90004D0406C07BDA80914D048F5F80934D0425
:101BA0008FE120904D048215A8F72090CF0330904C
:101BB000D0032220F1F43320E1F42090CC033090C4
:101BC000CD032220B1F43320A1F422242092080472
:101BD0002092090420920A0420920B040E942A02F7
:101BE00089EE95E09983888328E034E004E00E9440
:101BF0002B0222242092CE0333243092E60320923B
:101C0000E50316E0009147040E946B1E8EE1102F41
:101C1000082F0103009208040E942A0286EF95E033
:101C20009983888328E034E001E00E942B0222247B
:101C300020923C041EC02224209208042092090411
:101C40000E942A02A0903C042A2C3324822D99273A
:101C50008050994F2C01420C531C5982488228E035
:101C600034E002E00E942B0280913C048F5F80935D
:101C70003C0480913C04843BF0F2222420925604E0
:101C800020925304332430925504209254048091BE
:101C900038038F7D80933803309838988D7F8093F8
:101CA000380320925E0420925F0420925A0420920E
:101CB00059042092580488E780935B04209287049B
:101CC000309285042092840488E880933D048091BA
:101CD00038038064809338038F778093380384605F
:101CE00080933803877F80933803809137038B7FFD
:101CF00080933703877F809337038F7D80933703EB
:101D000080E98AB9809136038E7F80933603809173
:101D100035038D7F80933503809136038D7F8093CB
:101D200036038F7D809336038F7E80933603877FC3
:101D3000809336038B7F8093360380E981B9949832
:101D40002092930381B5886181BD8FE081BD789435
:101D50000C949B1CA89580913803817009F476C17E
:101D60008091370386958695817009F46FC18091C3
:101D700038038E7F8093380385E0209058048215C5
:101D800060F420905B04222041F48093580480E0AA
:101D900090E29093DC038093DB038FEF90E0209040
:101DA000DB033090DC038215930540F5AA9AAB98CB
:101DB00030923403209233032090340320923C0469
:101DC0000AC0809153048F5F80935304863018F0CB
:101DD0002224209253041091530401E00E94F21E29
:101DE00020903C04202269F3A09053048A2D8F5F39
:101DF000809353040A2D0E94D40628C12090DB034F
:101E00003090DC03222019F4332009F4A6C0AA98EC
:101E1000AB9A309234032092330320923C040AC0E0
:101E2000809153048F5F80935304863018F02224EE
:101E3000209253041091530401E00E94F21E20905E
:101E40003C04202269F382E020905304821558F468
:101E50008091DD039091DE038030E0E89E0718F06A
:101E600085E080935304A09053048A2D8F5F809364
:101E700053040A2D0E94060780912E038F5F8093E2
:101E80002E03843069F48091DD039091DE038F3F4F
:101E9000EFE79E0728F480912E038F5F80932E0337
:101EA0008AE020902E03821518F481E080932E039F
:101EB000A0902E03BB24C5018130E0E09E0729F1EC
:101EC0008230E0E09E0729F18330E0E09E0729F1AF
:101ED0008430E0E09E0729F18530E0E09E0729F19B
:101EE0008630E0E09E0729F18730E0E09E0729F187
:101EF0008830E0E09E0729F18930E0E09E0729F173
:101F00008A30E0E09E0729F1A1C001E00E9420058F
:101F10009DC001E00E94460599C001E00E9468054D
:101F200095C001E00E948E0591C001E00E94B405B9
:101F30008DC001E00E94D80589C001E00E94210601
:101F400085C001E00E94460681C001E00E9484062F
:101F50007DC001E00E94BD0679C0AA9AAB9A80912B
:101F60002E038F5FA82EA0922E0384E08A1518F40A
:101F7000222420922E03A0902E03BB24AA2011F429
:101F8000BB2091F0C5018130E0E09E07A1F08230D6
:101F9000E0E09E0719F18330E0E09E0731F18430E4
:101FA000E0E09E0749F152C000270E94200501E0B1
:101FB0000E9446054BC000270E9468058091DD0302
:101FC0009091DE038F3FEFE79E0720F401E00E942F
:101FD00044073CC001E00E948E0538C000270E94E3
:101FE000B40501E00E94D80531C000270E942106F7
:101FF00001E00E9446062AC08091360386958695A8
:10200000869586958695869586958170C9F021E09E
:1020100009E00E94F50220903F0425FE08C080914F
:1020200036038068809336030E9429070CC0809194
:10203000360380688093360300270E94840603C01D
:1020400000270E94840601E00E94BD0680913803AB
:102050008695817009F4EFC3159BEDC3A090C3036F
:10206000BB24C5018130E0E09E0709F42EC0823018
:10207000E0E09E0709F46AC08330E0E09E0709F4BF
:1020800028C18430E0E09E0709F483C18530E0E098
:102090009E0709F4DEC18630E0E09E0709F439C2EC
:1020A0008730E0E09E0709F48EC28B30E0E09E07A7
:1020B00009F4CAC28C30E0E09E0709F40AC38D30EF
:1020C000E0E09E0709F45DC3B4C320905E042220C3
:1020D00039F585E08093690388E080936A038091F5
:1020E00092038F7780936B0381E080936C0388E089
:1020F00080936D0380936E0304E610E00E949F1CA2
:10210000A0905E04BB248A2D8F5F80935E0489E6D5
:1021100093E0EA2DFF27E80FF91F208023B88BC337
:1021200080915E04863078F489E693E0E0915E0465
:10213000FF27E80FF91F208023B880915E048F5F8E
:1021400080935E0478C30E949D1D75C320905E0439
:10215000222009F0A9C085E08093690388E080937C
:102160006A0382E080936B038CE180936C03209080
:10217000650420926D032090670420926E03809185
:1021800066048F70829520906804282A20926F033D
:10219000209069042092700320906B0420927103B8
:1021A00020906C042092720320906D04209273039F
:1021B00020906E042092740320906F042092750387
:1021C000209071042092760320907204209277036D
:1021D0002090730420927803209079042092790350
:1021E00020907A0420927A0320917C04332700E027
:1021F00011E00E94831E20907B043324200E311EA8
:102200002AE030E081010E94CB1D00937B032090E7
:102210007D0420927C0320907F0420927D032090F7
:10222000910320927E032090920320927F032090BE
:1022300095032092800320909603209281032090A2
:10224000970320928203209098032092830320908A
:1022500099032092840320909B0320928503209071
:102260009C032092860320909D0320928703209058
:102270009E03209288030E94DA08A02EA092890370
:1022800004E610E00E949F1CA0905E04BB248A2DEF
:102290008F5F80935E0489E693E0EA2DFF27E80FC5
:1022A000F91F208023B8C7C280915E04813270F488
:1022B000A82EBB248F5F80935E0489E693E0EA2D0D
:1022C000FF27E80FF91F208023B8B5C20E949D1D8B
:1022D000B2C220905E04222009F042C085E08093C3
:1022E000690388E080936A0384E880936B0388E144
:1022F00080936C03222420923C0415C0A0903C04DF
:1023000081E993E0EA2DFF27E80FF91F20808DE691
:1023100093E0EA2DFF27E80FF91F208280913C040B
:102320008F5F80933C0480913C04883138F30E9495
:10233000DA08A02EA092850304E610E00E949F1CFC
:10234000A0905E04BB248A2D8F5F80935E0489E693
:1023500093E0EA2DFF27E80FF91F208023B86BC216
:1023600080915E048D3170F4A82EBB248F5F809322
:102370005E0489E693E0EA2DFF27E80FF91F20802D
:1023800023B859C2222420925E048CE08093C303B8
:1023900052C220905E04222009F042C085E0809362
:1023A000690388E080936A0388E880936B038CE17B
:1023B00080936C03222420923C0415C0A0903C041E
:1023C00081E993E0EA2DFF27E80FF91F20808DE6D1
:1023D00093E0EA2DFF27E80FF91F208280913C044B
:1023E0008F5F80933C0480913C048C3138F30E94D1
:1023F000DA08A02EA092890304E610E00E949F1C38
:10240000A0905E04BB248A2D8F5F80935E0489E6D2
:1024100093E0EA2DFF27E80FF91F208023B80BC2B5
:1024200080915E04813270F4A82EBB248F5F80936C
:102430005E0489E693E0EA2DFF27E80FF91F20806C
:1024400023B8F9C1222420925E048BE08093C30359
:10245000F2C120905E04222009F042C085E0809302
:10246000690388E080936A0380E980936B0388E1C5
:1024700080936C03222420923C0415C0A0903C045D
:1024800081E993E0EA2DFF27E80FF91F20808DE610
:1024900093E0EA2DFF27E80FF91F208280913C048A
:1024A0008F5F80933C0480913C04883138F30E9414
:1024B000DA08A02EA092850304E610E00E949F1C7B
:1024C000A0905E04BB248A2D8F5F80935E0489E612
:1024D00093E0EA2DFF27E80FF91F208023B8ABC156
:1024E00080915E048D3170F4A82EBB248F5F8093A1
:1024F0005E0489E693E0EA2DFF27E80FF91F2080AC
:1025000023B899C1222420925E048DE08093C303F6
:1025100092C120905E04222009F03FC085E08093A4
:10252000690388E080936A03809192038F77809398
:102530006B0386E080936C032090910320926D03DF
:102540002090920320926E032090930320926F03B9
:1025500020909403209270032090950320927103A1
:1025600020909603209272030E94DA08A02EA09277
:10257000730304E610E00E949F1CA0905E04BB243D
:102580008A2D8F5F80935E0489E693E0EA2DFF2712
:10259000E80FF91F208023B84EC180915E048B3074
:1025A00078F489E693E0E0915E04FF27E80FF91FD5
:1025B000208023B880915E048F5F80935E043BC1CE
:1025C0000E949D1D38C120905E04222039F585E0CF
:1025D0008093690388E080936A03809192038F77E8
:1025E00080936B0381E080936C0387E080936D039D
:1025F00080936E0304E610E00E949F1CA0905E048E
:10260000BB248A2D8F5F80935E0489E693E0EA2DD8
:10261000FF27E80FF91F208023B80DC180915E04C9
:10262000863078F489E693E0E0915E04FF27E80FB6
:10263000F91F208023B880915E048F5F80935E0431
:10264000FAC00E949D1DF7C020905E04222061F513
:1026500085E08093690388E080936A0380936B032D
:1026600083E080936C032090AD0320926D03209053
:10267000AE0320926E032090AF0320926F030E945E
:10268000DA08A02EA0927003A0905E04BB248A2DCD
:102690008F5F80935E0489E693E0EA2DFF27E80FC1
:1026A000F91F208023B8C7C080915E04883070F481
:1026B000A82EBB248F5F80935E0489E693E0EA2D09
:1026C000FF27E80FF91F208023B8B5C00E949D1D89
:1026D000B2C020905E04222009F03EC085E08093C5
:1026E000690388E080936A0384E080936B0388E148
:1026F00080936C03222420923C0415C0A0903C04DB
:1027000089EA93E0EA2DFF27E80FF91F20808DE684
:1027100093E0EA2DFF27E80FF91F208280913C0407
:102720008F5F80933C0480913C04883138F30E9491
:10273000DA08A02EA0928503A0905E04BB248A2D07
:102740008F5F80935E0489E693E0EA2DFF27E80F10
:10275000F91F208023B86FC080915E048D3170F422
:10276000A82EBB248F5F80935E0489E693E0EA2D58
:10277000FF27E80FF91F208023B85DC00E949D1D30
:102780005AC020905E04222009F03EC085E080936C
:10279000690388E080936A0380E180936B0388E19A
:1027A00080936C03222420923C0415C0A0903C042A
:1027B00089EA93E0EA2DFF27E80FF91F20808DE6D4
:1027C00093E0EA2DFF27E80FF91F208280913C0457
:1027D0008F5F80933C0480913C04883138F30E94E1
:1027E000DA08A02EA0928503A0905E04BB248A2D57
:1027F0008F5F80935E0489E693E0EA2DFF27E80F60
:10280000F91F208023B817C080915E048D3170F4C9
:10281000A82EBB248F5F80935E0489E693E0EA2DA7
:10282000FF27E80FF91F208023B805C00E949D1DD7
:1028300002C00E949D1D80913803869586958695DD
:10284000817009F43FC222242092830482E08093A5
:102850003C0412C081E694E0E0913C04FF27E80FBD
:10286000F91F208030908304320C309283048091D1
:102870003C048F5F80933C0480913C04803250F391
:102880008091370384608093370322242092580478
:102890002090810430908304321409F00BC2209000
:1028A0006304209233032090640420923403209028
:1028B0003303309034033092FC032092FB032090CA
:1028C0006504209233032090660420923403209004
:1028D0003303309034033092FA032092F9032090AE
:1028E00067042092330320906804209234032090E0
:1028F0003303309034033092F8032092F703209092
:1029000069042092330320906A04209234032090BB
:102910003303309034033092F6032092F503209075
:102920006B042092330320906C0420923403209097
:102930003303309034033092F4032092F303209059
:102940006D042092330320906E0420923403209073
:102950003303309034033092F2032092F10320903D
:102960006F0420923303209070042092340320904F
:102970003303309034033092EE032092ED03209025
:10298000710420923303209072042092340320902B
:102990003303309034033092F0032092EF03209001
:1029A0007304209233032090740420923403209007
:1029B0003303309034033092EC032092EB032090E9
:1029C00075042092330320907604209234032090E3
:1029D0003303309034033092EA032092E9032090CD
:1029E00077042092330320907804209234032090BF
:1029F0003303309034033092E8032092E7032090B1
:102A00007B042092330320907C0420923403209096
:102A10003303309034033092E0032092DF0380E8E8
:102A200020907D04821538F4809137038062809372
:102A30003703A99806C0809137038F7D80933703B1
:102A4000A99A20907D042092330320907E04209246
:102A5000340320903303309034033092DE0320920D
:102A6000DD0320907D0426FE09C08091DD03909156
:102A7000DE0390689093DE038093DD0380917F04F2
:102A80008F7180933303809180048F71809334031E
:102A900020903303309034033092DC032092DB0328
:102AA000A090DB03B090DC032090540430905504D8
:102AB0002A143B0471F0AA2011F4BB2051F080913C
:102AC00038038062809338031501309255042092B8
:102AD0005404209079042092330320907A042092A9
:102AE00034032AE030E000913303109134030E9454
:102AF000E71D1093E6030093E50321E006EF15E0E0
:102B00000E94AE0220900804209239042090E50330
:102B10003090E6033092340320923303209208046D
:102B200020903403209209040E942A022090390444
:102B30003324822D99278050994F2C01420C531C2D
:102B40005982488228E034E002E00E942B02809102
:102B500039048F5F809308040E942A0286EF95E073
:102B60009983888328E034E001E00E942B02809161
:102B70003603817009F46AC0809136038E7F80939A
:102B800036038091350381608093350386E080931E
:102B9000860488E08AB9222420925E0481EF809323
:102BA00091038093920388E0809393032090FE0327
:102BB000209294032090FF0320929503209000041C
:102BC0002092960320900104209297032090020403
:102BD00020929803209003042092990320900404EB
:102BE00020929A032090050420929B032090FF03DB
:102BF0003090FE03320C20900004320C209001042F
:102C0000320C20900204320C20900304320C2090ED
:102C10000404320C20900504320C30929C0310C046
:102C20005D9B0EC081E993E0E0915E04FF27E80F11
:102C3000F91F20802CB880915E048F5F80935E0422
:102C400080915E048C3060F380E98AB9809135030D
:102C5000817081F120908604222061F1822D8150C3
:102C600080938604882339F4809135038E7F809386
:102C700035030E949D1D80916204813711F08135DA
:102C8000C9F480916204813731F480913503846006
:102C90008093350305C0809135038B7F8093350386
:102CA0000E949D1D809135038E7F80933503826045
:102CB0008093350380913803846080933803877F45
:102CC000809338038091380382958F70817009F466
:102CD000FBC10E94C808809138038F7E809338031F
:102CE00080E08093E1038093E2038093E303809389
:102CF000E40321E006EF15E00E94AE0220900804F4
:102D00002092390484EB821510F480933904222434
:102D100020923C0434C022E0A0903C042A2C3324AE
:102D2000022D11270050194F020D131D0E94AE02F3
:102D30002090080420923303209009042092340349
:102D40002090330330903403442455248090E303CF
:102D50009090E4036090E1037090E203620C731CB6
:102D6000841C951C7092E2036092E1039092E4034C
:102D70008092E30380913C048F5F80933C04209019
:102D80003904332440903C045524241435041CF6A3
:102D900044EB50E060E070E02091E3033091E40305
:102DA0000091E1031091E2037A936A935A934A9354
:102DB0000E94011E1093E6030093E5032224209253
:102DC00008040E942A0286EF95E09983888328E010
:102DD00034E001E00E942B022090E5033090E603EE
:102DE0004090CA035090CB03420C531C5092CB032B
:102DF0004092CA034090C8035090C903420C531C30
:102E00005092C9034092C80328EE33E00091CA03F0
:102E10001091CB030E94E71D00933C04202E002359
:102E200009F470C033244090CC035090CD03420C81
:102E3000531C5092CD034092CC03222D332708EE31
:102E400013E00E94831E2090CA033090CB03201A07
:102E5000310A3092CB032092CA0320903C04309078
:102E6000D603320C3092D6031AE0032D0E946D1E59
:102E7000002309F447C08091D6038A508093D6037B
:102E800041E050E060E070E04090D9035090DA03F8
:102E90002090D7033090D803240E351E461E571EAF
:102EA0003092D8032092D7035092DA034092D9038C
:102EB00040EE53E964E070E02416350646065706F6
:102EC00048F080E08093D7038093D8038093D903A0
:102ED0008093DA0341E050E060E070E04090C60388
:102EE0005090C7032090C4033090C503240E351EB4
:102EF000461E571E3092C5032092C4035092C7034A
:102F00004092C6038091CF039091D0030196909395
:102F1000D0038093CF038091D1038F5F8093D1033F
:102F200041E050E060E070E04090D4035090D50361
:102F30002090D2033090D303240E351E461E571E18
:102F40003092D3032092D2035092D5034092D403FF
:102F500089E02090D103821518F422242092D10315
:102F60004090D9035090DA032090D7033090D803D3
:102F70003092300320922F0350923203409231035B
:102F800020920804209030032092090420903103FD
:102F900020920A042090320320920B042090D60342
:102FA00020920C044090D4035090D5032090D2037B
:102FB0003090D3033092300320922F03509232038B
:102FC0004092310320920D042090300320920E0491
:102FD0002090310320920F0420903203209210049D
:102FE0002090CF033090D0033092340320923303EB
:102FF0002092110420903403209212042090CC03DC
:103000003090CD0330923403209233032092130486
:1030100020903403209214042090CA033090CB03F4
:10302000309234032092330320921504209034030D
:10303000209216042090C8033090C90330923403C4
:103040002092330320921704209034032092180416
:103050002090D103209219044090C6035090C703DA
:103060002090C4033090C5033092300320922F0388
:10307000509232034092310320921A042090300380
:1030800020921B042090310320921C0420903203D4
:1030900020921D0426E003E00E94F502F8940E94AD
:1030A0002A0280EE95E09983888328E034E006E1E7
:1030B0000E942B0222243324398228822FE334E019
:1030C00006E00E942B0278942899D4C0809137039F
:1030D00086958695817009F4CDC00E94C8088091BC
:1030E00057048F5F8093570481E020905704821526
:1030F00028F4809136038D7F8093360326E003E029
:103100000E94F50220903F04209248042090400441
:1031100020924B042090420420924E0420904304BD
:1031200020925004209044042092510400914804BD
:103130000E94A808A02E2090CE033A2C320C309288
:103140003C04A0903D048A2D883821F0232C821560
:1031500009F490C020903C0420923D0416E0022D1A
:103160000E946B1E002329F48091380380618093B4
:10317000380380914B04833259F480914804893597
:1031800039F400914E040E94A808A02EA0924C048D
:1031900020904804222009F06DC000914B040E9449
:1031A000A808A02EA092490400914E040E94A808ED
:1031B000A02EA0924D040E940408209049042220D1
:1031C00009F052C020904C0420924D040E94460801
:1031D0000E940408222433243092C9032092C80399
:1031E0003092CD032092CC033092D0032092CF03B3
:1031F00000914E040E94A808A02EA0924D04222403
:103200002092490407C00E940408809149048F5FFE
:1032100080934904809149048831A8F322242092A4
:10322000490480914E048130F9F4009150040E94C9
:10323000A808A02EA0924F04013021F48CE08093C6
:103240004F0405C080914F04815080934F0400913A
:103250004F040E946A0880E08093C4038093C503F2
:103260008093C6038093C703222433243092C9037A
:103270002092C803A09038038A2D8695869586955E
:103280008695869586958695817009F4D9C28A2D92
:1032900086958170809509F4D3C28A2D8F778093AB
:1032A000380322242092C20320923C0412C081E9F8
:1032B00093E0E0913C04FF27E80FF91F2080309055
:1032C000C203320C3092C20380913C048F5F809322
:1032D0003C0480915F04815020903C04281638F310
:1032E00080E993E0E0915F04FF27E80FF91F208059
:1032F0003090C203321409F09BC2809192038A3A43
:1033000009F480C280919203823C39F585E02090D7
:103310005B048215D8F42090940320920804209036
:103320009503209209042090960320920A040E949B
:103330002A0286E09FE19983888328E034E003E055
:103340000E942B0281E08093C30303C087E0809337
:10335000C30382E48093930355C280919203813C1E
:1033600059F585E020905B048215F8F420909403D1
:10337000209208042090950320920904209096033F
:1033800020920A042090970320920B040E942A02A4
:1033900089E09FE19983888328E034E004E00E947B
:1033A0002B0281E08093C30303C087E08093C303B3
:1033B00081E48093930326C280919203803C09F0BC
:1033C0004BC08091350386958170A1F080913503C3
:1033D0008D7F8093350386958695817021F081E0FD
:1033E0008093C30303C087E08093C30380E480938A
:1033F000930308C2809136038170813049F1809136
:103400003603816080933603209094032092FE035C
:10341000209095032092FF032090960320920004B1
:103420002090970320920104209098032092020498
:10343000209099032092030420909A032092040480
:1034400020909B032092050422242092C303DAC11A
:1034500022242092C303D6C180919203813809F0BF
:103460003BC0222420923C0415C0A0903C0484E977
:1034700093E0EA2DFF27E80FF91F20808FE394E007
:10348000EA2DFF27E80FF91F208280913C048F5F0F
:1034900080933C0480913C04873038F327E002E0BD
:1034A0000E947F0220904004209248042090410412
:1034B00020924B042090430420924E042090440418
:1034C00020925004209045042092510481E0809382
:1034D00093038093C30396C180919203823009F0D5
:1034E0006AC02090CC033090CD0344245524309200
:1034F000300320922F0350923203409231032092E6
:103500009103209030032092920320903103209267
:10351000930320903203209294034090D90350905B
:10352000DA032090D7033090D803309230032092F2
:103530002F03509232034092310320929503209042
:10354000300320929603209031032092970320901D
:103550003203209298032090CF033090D003309212
:103560003403209233032092990320903403209255
:103570009A034090D4035090D5032090D20330900A
:10358000D3033092300320922F03509232034092A3
:10359000310320929B032090300320929C032090C3
:1035A000310320929D032090320320929E0382E0FB
:1035B0008093C30327C180919203843009F064C0D3
:1035C000209094032092C203022D0E94A808A02EEE
:1035D00000E31A2D0103C001C09790933B04809330
:1035E0003A0420E38C010E94AE02222420923C0483
:1035F00015C0A0903C0488E094E0EA2DFF27E80F76
:10360000F91F208081E993E0EA2DFF27E80FF91FD9
:10361000208280913C048F5F80933C0480913C0425
:10362000803338F32090C20330904E04321441F5B9
:103630002090C8033090C9033092340320923303A2
:1036400000914B040E94A808A02E81E993E0EA2D86
:10365000FF27EE0FFF1FE80FF91F20903303208292
:1036600000914B040E94A808A02E82E993E0EA2D65
:10367000FF27EE0FFF1FE80FF91F20903403208271
:1036800083E08093C303BEC080919203883041F5EC
:103690000E9446082FE100E016E00E94AE022224BC
:1036A00020923C0415C0A0903C0488E094E0EA2DF0
:1036B000FF27E80FF91F208081E993E0EA2DFF271B
:1036C000E80FF91F208280913C048F5F80933C04B7
:1036D00080913C048F3138F384E08093C30392C01F
:1036E00080919203803179F5009150040E94A808DE
:1036F000A02EA0924F040E946A0820E300E916E081
:103700000E94AE02222420923C0415C0A0903C04EA
:1037100088E094E0EA2DFF27E80FF91F208081E977
:1037200093E0EA2DFF27E80FF91F208280913C04E7
:103730008F5F80933C0480913C04803338F385E0B4
:103740008093C3035FC080919203803209F04EC022
:103750002090940320923303209095032092340309
:10376000209133033091340305E010E00E94831E62
:10377000C8018052964F909334038093330388E6B8
:103780009DE120903303309034038215930530F48B
:1037900080EE99E0909334038093330326E0009108
:1037A0003303109134030E94AE02222420923C0481
:1037B00015C0A0903C0488E094E0EA2DFF27E80FB4
:1037C000F91F208081E993E0EA2DFF27E80FF91F18
:1037D000208280913C048F5F80933C0480913C0464
:1037E000863038F386E08093C3030CC08091920347
:1037F000833441F48091360382608093360322241F
:103800002092C3032090C303222061F0222420923F
:103810005E048091380382608093380388E081B928
:10382000949A0EC08091380380648093380308C056
:1038300080913803806480933803222420925F04AF
:1038400080913803869586958695869586958170B4
:1038500009F464C0809138038F7D8093380322E09F
:1038600007EF15E00E94AE02209008042092330377
:1038700020900904209234032090480420920804E8
:1038800020904B042092090420904E0420920A04B8
:103890002090540430905504232C332420920B04A0
:1038A000209054043090550420920C040E942A0267
:1038B00020903303309034033982288228E034E0AA
:1038C00005E00E942B0280913303909134038836E7
:1038D000EDE19E0738F080EE99E0909334038093F9
:1038E000330309C08091330390913403059690937C
:1038F00034038093330320903303209208042090F4
:103900003403209209040E942A0287EF95E09983EC
:10391000888328E034E002E00E942B028091370384
:1039200082958F70817039F0809137038F7E8093FC
:1039300037030E949D1D0C94AA0E229608954A9367
:103940005A9309C04427552702C04F5F5F4F403A42
:10395000E0E05E07D0F3180101501040222091F7FB
:10396000332081F75991499108952A923A928A9386
:103970009A93EA93FA932FB62A9220903803822DD5
:10398000869586958170C1F0822D8695869586955F
:10399000817091F42CB020926104822D813F09F056
:1039A00051C0809138038B7F8093380381E08093EE
:1039B000600480935A0446C08091380386958695AA
:1039C0008695817009F03EC0809160048130B1F429
:1039D0002CB02092620482E08093600480916104A4
:1039E000813F81F180913803877F80933803846021
:1039F00080933803222420925A0424C080916004CA
:103A0000813278F481E694E0E0916004FF27E80FCA
:103A1000F91F2CB02082809160048F5F8093600436
:103A200011C08091380388608093380381E694E068
:103A3000E0916004FF27E80FF91F2CB020822224B8
:103A400020925A0429902FBEF991E9919991899178
:103A50003990299018958898899A919A8FE589B913
:103A6000222420BC2BB82AB886E880BD08952A926B
:103A70006A928A939A93EA93FA932FB62A92809144
:103A80003803869586958695869586958695817068
:103A9000C9F080915F048230A8F423B02092910392
:103AA000822D8A3A09F034C0809138038F7B80934D
:103AB000380380915F048F5F80935F0481E080937F
:103AC000590426C0809193038C5F20905F042816D0
:103AD00070F480E993E0E22DFF27E80FF91F23B08F
:103AE000208280915F048F5F80935F0411C080917A
:103AF000380380688093380380E993E0E0915F04A5
:103B0000FF27E80FF91F23B02082222420925904B6
:103B100029902FBEF991E991999189916990299005
:103B20001895BA98BB9A8FE580B922242CBE22B88A
:103B300080E881B986E88CBF08950027112704C06A
:103B4000000000000F5F1F4F0038E6E01E07C0F3C3
:103B5000222420929303809138038D7F8093380331
:103B600088E081B9949A80E482B980E981B9949817
:103B700020925F042092C303809138038064809375
:103B8000380308953A932A931A930A9308956894F0
:103B9000DA92D12E04C0E894DA92D12ED32617FF00
:103BA00004C0109500950F5F1F4F37FF04C030957C
:103BB00020952F5F3F4F0E94E81DD7FE04C010954F
:103BC00000950F5F1F4FD9900895689401C0E89445
:103BD000EA92FA928A93EE24FF2480E1000F111FEB
:103BE000EE1CFF1CE216F30618F0E21AF30A039526
:103BF0008A95A1F716F40E2D1F2D8991F990E99061
:103C00000895E89401C0689430D0CC2409C0E894A9
:103C100001C068942AD037FD0E94E91EB7FD52D03A
:103C2000772488249924AA24BB2442D0C1F045D00B
:103C3000B1F0E8E2000F111F221F331F771C881C10
:103C4000991CAA1CBB1C88169906AA06BB0628F05C
:103C5000881A990AAA0ABB0A0395EA9559F726F425
:103C6000082D192D2A2D3B2D13C07A928A929A92F3
:103C7000AA92BA92CA92EA938A939A93AA93BA930F
:103C80008B859C85AD85BE85C32E0EF0CB26089511
:103C9000C7FC0E94E91EB991A99199918991E99176
:103CA000C990B990A9909990899079902496089597
:103CB000E02FE12BE22BE32B0895E82FE92BEA2BF1
:103CC000EB2B089580959095A095B0958F5F9F4FB1
:103CD000AF4FBF4F0895689401C0E8942A93FA92B9
:103CE000EA92FF24EE2420E1000FFF1CEE1CE116F7
:103CF00010F0E11A03952A95B9F70EF40E2DE9900C
:103D0000F990299108950A921A928A939A93029FA0
:103D1000C001129F900D039F900D8C019991899184
:103D2000199009900895A990B990C990D990E990F7
:103D3000F9904991599108957A936A935A934A93C5
:103D4000FA92EA92DA92CA92BA92AA9208955A9391
:103D50004A93BA92AA920895A990B990499159911B
:103D600008957A936A935A934A9308954991599181
:103D70006991799108957A936A935A934A93BA9282
:103D8000AA920895A990B990499159916991799110
:103D900008955A934A93DA92CA92BA92AA920895CF
:103DA000A990B990C990D9904991599108957A9361
:103DB0006A935A934A93DA92CA92BA92AA9208954F
:103DC000A990B990C990D9904991599169917991E7
:103DD000089500951095209530950F5F1F4F2F4F38
:103DE0003F4F0895112319F0000F1A95FBCF089546
:103DF000FFFFFFFFFFFFFFFFFFFFFFFFFFFFFFFFD3
:103E0000FFFFFFFFFFFFFFFFFFFFFFFFFFFFFFFFC2
:103E1000FFFFFFFFFFFFFFFFFFFFFFFFFFFFFFFFB2
:103E2000FFFFFFFFFFFFFFFFFFFFFFFFFFFFFFFFA2
:00000001FF
